:100000000C94E8000C9477090C9405010C940501FC
:100010000C9405010C9405010C9405010C94050148
:100020000C9405010C9405010C9405010C94050138
:100030000C9405010C9405010C9405010C94050128
:100040000C9405010C9405010C9405010C94050118
:100050000C9405010C9405010C9405010C94050108
:100060000C9405010C9405010C9405010C940501F8
:100070000C9405010C9405010C940501CB05CD05EC
:10008000D005D205D505D705DA05DC05DF05E10584
:10009000E305E605E805EA05EC05EE05F005F205E1
:1000A000F4056706670667066706F605F805FA05AC
:1000B000FC056706670667066706FE05000602067A
:1000C0000406060608060A060C060E0610061206A8
:1000D0001406160618061A061C0667066706670643
:1000E00067061E06200665062206240628062B063D
:1000F0002F063206380635063106340637063A062C
:100100003C063E06400642064406460648064A06A7
:100110004C064E06500652065406560658065A0617
:100120005C06670667066706670661065E06600688
:1001300064067406780676067A06800687068906BF
:100140008B068D0697069A06EE06F006F206F40672
:10015000F606F806FA06FC06FE0600070207060782
:10016000090212000101008096090400000000004D
:10017000000012011001FF000008C016DC0500029B
:10018000010200011E0349004E004C0020005200F5
:100190006500740072006F002D00500072006F0047
:1001A00067002A0349006E00660069006E0069005E
:1001B000740065004E00650073004C006900760015
:1001C000650073002E0063006F006D0004030904D6
:1001D00011241FBECFEFD4E0DEBFCDBF11E0A0E001
:1001E000B1E0ECE6F5E102C005900D92A230B10756
:1001F000D9F713E0A2E0B1E001C01D92AD38B1071C
:10020000E1F70E948B0A0C94B40A0C940000CF9280
:10021000DF92EF92FF92CF93DF93DB01F701E601CC
:10022000813579F1F0F4803509F04BC012968C914C
:100230001297808313968C911397818314968C91D7
:100240001497828315968C911597838316968C91BB
:100250001697848317968C911797858318968C919F
:100260002AC0803629F0813661F58091300105C0C1
:10027000A22FB0E0AF5ABE4F8C91808388818F5FF0
:100280001DC019968C91199780831A968C911A9794
:1002900081831B968C911B9782831C968C911C9753
:1002A00083831D968C911D9784831E968C911E9737
:1002B00085831F968C9186838881895F888380E0FF
:1002C00001C084EBDF91CF91FF90EF90DF90CF9052
:1002D0000895CF93DF93FC01DB01E9018091410197
:1002E0009091420120812078203849F4368138836A
:1002F000442309F445C08D919C9111970CC02FEFB8
:100300002883268120932F01442351F170936203A7
:100310006093610320E913962C93139714961C9213
:100320002281213711F02034F1F5A0916103B091C1
:1003300062030D90BC91A02D25812C93A0916103A7
:10034000B09162030D90BC91A02D248111962C9345
:10035000E0916103F091620324812E5F248323C026
:10036000A0911D01B0911E01B0936203A09361039F
:1003700020E913962C93A0911D01B0911E01CECFC0
:10038000A0911D01B0911E0113963C911397383D29
:1003900021F48D919C911197ECCF2FEF288320E1D0
:1003A00020933001E8CFDF91CF910895E1E5F1E0AE
:1003B0009FEF8FEF919321E0E136F207D1F7809321
:1003C000440180932201809347018093250180930B
:1003D000340180931001809337018093130181E0F1
:1003E000809330010895FB01803391F038F4882325
:1003F00061F08130B9F42093300112C0823371F082
:1004000050F0833379F427870BC00E94D60108C0CF
:100410004187228705C04387248702C045872687F6
:1004200080E0089584EB0895CF93DF93FC0150E0C2
:10043000CA01820F911D41970CF047C0222309F495
:1004400046C083818F3F09F044C086818F3F09F009
:1004500042C080E090E0EA01CF5ADE4F821750F4AC
:100460000196DE01A80FB91F11973C913F3FB1F3F0
:1004700081EC32C066831382822F8295880F807E42
:10048000815082831482158210861782118612860B
:1004900013861486158616861786CA0135E0880FDE
:1004A000991F3A95E1F78F599E4F9183808380E0A1
:1004B00090E04F5A5E4F821730F4FA01E80FF91FAF
:1004C00060830196F8CF80E007C08EEB05C082EC18
:1004D00003C08FEB01C080ECDF91CF9108950F93A3
:1004E000FB01642F422F202F803888F0883858F085
:1004F0008059883060F40583242F30E0362B308714
:10050000278380E005C0CF010F910C94140286EB85
:100510000F910895CF92DF92EF92FF920F93CF93B6
:10052000DF93FC01EB016A01828190ED980F90331B
:1005300070F49381913071F050F0923029F0933043
:10054000C1F56DE071E008C061E371E005C061E4F0
:1005500071E002C06FE171E0803768F4803580F4AB
:10056000803408F047C00381248145810E94F30153
:10057000888381E03CC0803868F4960140E03CC04C
:100580007E019FEFE91AF90A0381248145810E94C7
:1005900007013DC0982F97709130A1F080F0923004
:1005A00029F0933031F46DE071E00EC061E371E049
:1005B0000BC086E8888381E0D6018C9329C061E472
:1005C00071E002C06FE171E0803F50F4803C58F46C
:1005D0008038E0F00381248145810E946F0217C0BA
:1005E000883F40F013C0DB01CD91DC918681F6019C
:1005F00080830EC096014FEFCF01DF91CF910F9115
:10060000FF90EF90DF90CF900C94690185E888838C
:10061000CE01DF91CF910F91FF90EF90DF90CF90BF
:10062000089590914401809122018F3F29F481E047
:100630009F3F19F480E001C082E0909134019F3F18
:1006400009F083E0909110019F3F09F084E0089544
:10065000623049F421E08134920739F121E08F3191
:10066000920761F10895633069F421E081349207C3
:10067000E1F021E08F319207D9F021E08133920738
:10068000E9F008956430E1F421E08134920769F0E3
:1006900021E08F31920761F021E08133920759F018
:1006A00021E08D30920751F008958FE191E0089597
:1006B00081E391E008958DE091E0089581E491E077
:1006C0000895CF93DF93D09130018D2F8F7D823DA0
:1006D00001F50E941103C82F8093020121E431E04B
:1006E00030931E0120931D01D23D99F4C901D1E040
:1006F000DC1728F46C2F0E942803DF5FF9CF90935A
:100700001E0180931D0120E8FC01238380ED80936E
:10071000300180913001823F19F480EF80933001E5
:10072000C0913001C03D31F580911D0190911E01B5
:10073000FC0123812038F1F4609102010E9428031A
:1007400090931E0180931D01FC011482C3830E94BB
:10075000BD03E0911D01F0911E01882311F08383F8
:1007600009C088ED8383258187819085820F911D43
:1007700090878783DF91CF9108950F93CF93DF9375
:10078000EC016F8189858C3061F028F48A3039F072
:100790008B3081F002C08F3068F083EC0CC0606851
:1007A00001C060660FEF2A814E81888199810E9485
:1007B0008A058C8380E0DF91CF910F9108950F938C
:1007C0001F93CF93DF93EC011F8110689C818A8176
:1007D000981790F54AEA65E585E50E94B00445E57D
:1007E0006AEA8AE20E94B00440EA65E585E50E9473
:1007F000B0046C81E881F981E60FF11D4081812F01
:100800000E94B0046C81812F0E94D804082F6C8153
:10081000812F0E94D8040813F5CF8C81E881F981DB
:10082000E80FF11D9081091304C08F5F8C835998E4
:10083000CDCF519A599ACACF80E0DF91CF911F91C5
:100840000F91089511B88FEF82B914B885B917B810
:1008500088B98AB184718AB98BB18B6E8BB9509883
:1008600058985198599A08950E942204399A419AA9
:10087000389A40983A9A429A3C9A449A3D9A459AB4
:100880003F9A479A47988FEF84B915B8479A479887
:1008900014B812B881B914B885B908950E94220419
:1008A000399A419A3C9A449A3D9A459A509A589A54
:1008B0003F9A479A4798579A5F9A5F988FEF84B903
:1008C00015B8479A479814B884B915B85F9A5F98D5
:1008D00014B812B881B914B885B90895813049F0B7
:1008E00028F0823051F40E944E0405C00E94220478
:1008F00002C00E94340480E0089586E90895FC0156
:1009000081E080835898509A000089B18183509883
:100910005898908181818923891308C08AEA868347
:100920008483828385E58583838308955098589ACC
:1009300089B1818389B1828389B1838389B18483B9
:1009400089B1858389B186835098589808958038F5
:1009500029F4CB010E947F0480E0089587E908957F
:100960009FEF94B985B9479A479862B945B95898A5
:10097000509A5098589A14B808955098589840989A
:10098000419A429A62B99FEF94B985B9479A4798BC
:1009900014B800000000409A87FD41980000000054
:1009A000000000000000000083B14098419A0895C3
:1009B00062B99FEF94B985B9479A479814B8409A9D
:1009C00087FD4198000000000000000083B14098BE
:1009D000419A0895509858989FEF94B962B985B993
:1009E000479A4798429845B9409A87FD4198000038
:1009F00000004098419A429A14B808959FEF94B924
:100A0000803208F4806885B9479A479814B862B96B
:100A10004498000000000000000083B1449A08954B
:100A20009FEF94B9803208F4806885B9479A479857
:100A300062B945B9000045980000459A14B8089578
:100A4000982F862F642F422F913049F028F0923052
:100A500051F40E94EA0405C00E94B00402C00E9442
:100A6000100580E0089580EA08958FEF84B984E04E
:100A700085B9479A479829B188E085B9479A479838
:100A800089B1807214B891E0422F407225FD90E048
:100A900031E0882311F030E002C0911114C021E050
:100AA000411101C020E0811103C0222381F003C065
:100AB000222329F00AC0332351F082E108959923BB
:100AC00031F083E1089580E1089581E108958FEF89
:100AD0000895CF93DF93982F862F642FE9019138E3
:100AE00069F028F4903891F40E94BD040CC092384B
:100AF00041F0933859F40E94350505C00E94D8048E
:100B000002C00E94FE04888380E001C081EADF9178
:100B1000CF910895EF92FF920F93CF93DF9300D080
:100B20001F92CDB7DEB77C018FEF84B965B9479AC4
:100B3000479814B8409A67FD419842B980E0011186
:100B400003C00000000008C02B834A8389830E94F1
:100B50004E0889814A812B8193B1F701E80FF11D7D
:100B600090834F5F42B98F5F281748F74098419AAA
:100B70000F900F900F90DF91CF910F91FF90EF901A
:100B8000089590E08B35910508F0A1C0FC01E25C6E
:100B9000FF4F0C94AE0A11B895C08FEF81B992C087
:100BA00012B890C08FEF82B98DC014B88BC08FEF90
:100BB00084B988C015B886C08FEF85B983C017B8CF
:100BC00081C018B87FC08FEF88B97CC038987AC0D0
:100BD000389A78C0409876C0409A74C0399872C0EC
:100BE000399A70C041986EC0419A6CC03A986AC0F8
:100BF0003A9A68C0429866C0429A64C03B9862C004
:100C00003B9A60C043985EC0439A5CC03C985AC00F
:100C10003C9A58C0449856C0449A54C03D9852C01B
:100C20003D9A50C045984EC0459A4CC03E984AC027
:100C30003E9A48C0469846C0469A44C03F9842C033
:100C40003F9A40C0479A3EC08AB184718AB93AC07F
:100C50008BB1847102C08BB18B6E8BB933C050984D
:100C600031C05898509A2EC05098589A2BC050981E
:100C7000589828C0519826C0519A24C0599822C02B
:100C8000599A20C053981EC0539A1CC05B981AC032
:100C90005B9A18C0559816C0559A14C05D9812C03A
:100CA0005D9A10C056980EC0569A0CC05E980AC045
:100CB0005E9A08C0579806C0579A04C05F9A02C04F
:100CC0005F9A5F9880E00895479A4798FBCF8CE839
:100CD000089590E0FC01E058F109EB30F105A0F532
:100CE000E756FF4F0C94AE0A62B922C08FEF84B969
:100CF00065B91EC08FEF84B965B9479A479805C09A
:100D00008FEF84B965B95F9A5F9814B811C061B963
:100D10000FC064B90DC067B90BC09AB1862F84614A
:100D200089238AB98AB16B7E682B6AB901C068B918
:100D300080E008959BB1862F846189238BB98BB1A4
:100D40006B7E682B6BB9F4CF8DE80895813A61F022
:100D5000823AB9F0803A11F58FEF84B965B9479AB4
:100D6000479814B842B916C08FEF84B965B9479A4D
:100D7000479814B842B967FF02C041980BC0419A26
:100D800009C042B98FEF84B9603230F415B8479A80
:100D9000479814B880E0089565B9F9CF8EE80895B2
:100DA000803B61F422B98FEF84B945B9479A4798DF
:100DB00065B95F9A5F9814B880E008958FE8089548
:100DC000CF93DF93EB0190E0805C91098C3091052B
:100DD000F8F48C559F4FFC010C94AE0A80B113C0FF
:100DE00083B111C086B10FC089B10DC082B10BC0F3
:100DF00085B109C088B107C08BB105C081B103C0FE
:100E000084B101C087B1888380E003C08AB1FBCF81
:100E100080E9DF91CF9108950F93811102C0589A14
:100E200001C058988FEF84B922B945B9479A4798BD
:100E300005B9459800000000459A419A14B85898A1
:100E40000F9108950F93022F813061F030F08230BE
:100E500089F4242F462F60E008C0242F462F6FEF1F
:100E600081E004C0242F462F6FEF80E00E940C0722
:100E700080E001C08AEA0F9108950F93811102C0AA
:100E8000589A01C058988FEF84B902B925B9479A8A
:100E9000479845B95F9A5F9814B8449800000000DD
:100EA0000000000083B1449A419A58980F91089528
:100EB0000F931F93CF93DF93E801813851F082386D
:100EC00091F08038A9F4022F242F462F6FEF81E094
:100ED00005C0022F242F462F6FEF80E00E943D07B0
:100EE000888380E006C0022F242F462F60E0F5CFD4
:100EF0008BEADF91CF911F910F9108950F931F936C
:100F0000CF93DF931F92CDB7DEB7FC0183E091E072
:100F100090937203809371031982808187FF02C0CE
:100F200081E089838181833009F44BC028F48130CA
:100F3000D1F08230C1F179C0853009F467C008F47E
:100F400054C0863009F071C01092030180910B01EA
:100F500080930401E0916103F091620382818093A8
:100F6000050183E060C08281803B38F4803A88F4D8
:100F7000803858F40E94C10559C0803C78F424811F
:100F8000458163810E94D00651C064810E94690638
:100F90004DC0448165810E94A60648C064E071E0AE
:100FA0000E94E0061DC08281803818F40E946E0401
:100FB0003DC064E071E00E94A7048093030188E0D3
:100FC00032C08281803830F42381448165810E945F
:100FD00020052CC024E031E0448165810E94690530
:100FE0008093030189818F5F1EC08281803830F435
:100FF0002381448165810E94220718C004E011E02A
:101000002481458163810E945807EACFAE014F5F7A
:101010005F4F63E071E0CF010E948A0290937203F8
:101020008093710305C0898303C080E88093030126
:1010300089810F90DF91CF911F910F910895E091D9
:101040006103F0916203448120813181582FFC01BA
:10105000742F781B972F9E0F8E2F851B861730F4C9
:101060008191D901A90FB11D8C93F4CFE091610357
:10107000F09162038481860F848390912F01961BE7
:1010800090932F0110920B01640F8281861302C08E
:1010900088E9838381E0911180E00895CF93DF9305
:1010A00060917303635067FDA4C080917003CCE02E
:1010B000D0E0C81BD109C958DC4F80916F038D3235
:1010C00009F085C0683009F092C083EC8093630317
:1010D0008AE58093010110920C018881807621F0CD
:1010E000CE010E947E0760C08A8110926C039981B4
:1010F000911106C010926D032CE633E082E050C0DF
:10110000953019F4809374033DC09630A9F59B8106
:10111000913019F482E791E004C0923041F480E606
:1011200091E0909372038093710382E121C0933028
:10113000F1F4811108C08CEC91E0909372038093DC
:10114000710384E015C0813041F482EA91E090930C
:101150007203809371038AE20BC0823041F484E809
:1011600091E090937203809371038EE101C080E05F
:1011700090E490930C0118C0983079F0993031F4D4
:10118000809376032CE633E080E00AC081E09A3059
:1011900009F080E02CE633E003C026E733E081E08D
:1011A00030937203209371038F3F39F4988197FD38
:1011B0008E8190E890930C0107C09F81911104C02B
:1011C0009E81981708F4892F8093000110C08091A8
:1011D0000C0187FF0CC0CE010E941F088F3F21F435
:1011E0008EE18093010103C08111109200011092E1
:1011F00073038091010184FF4DC0809100018F3FF6
:1012000009F448C0C82F893008F0C8E08C1B8093CF
:1012100000018091630398E8892780936303CC23BE
:1012200061F1809171039091720320910C0126FF6E
:1012300012C0A4E6B3E023E633E020953095280FF2
:10124000391F4C2F4A0FF901EA0FFB1FE491ED9370
:101250004A13F9CF09C0E4E6F3E0DC012C2F2E0F8E
:101260003D9131932E13FCCF01962FEF2C0F820F5F
:10127000911D90937203809371036C2F84E693E029
:101280000E947309CC5FCC3019F08FEF809300017E
:10129000C093010184E199B1947131F48150D9F77F
:1012A0001092740310926E03DF91CF910895E9E6D6
:1012B000F0E0808182608083E89A0895A82FB92F9A
:1012C00080E090E041E050EA609530E009C02D9167
:1012D00082279795879510F084279527305EC8F36D
:1012E0006F5FA8F30895EADF8D939D930895CF93E0
:1012F000CFB7CF93DF93C3954C9BE9F74C9B0BC0C3
:101300004C9B09C04C9B07C04C9B05C04C9B03C029
:101310004C9B01C089C06F93C0917003DD27C958F1
:10132000DC4F2F9365E54C9B03C02F916F91E6CF67
:101330000F931F934F9320E040E15F9309B1047135
:1013400004FB27F93F9350E03BE039C0147140643F
:101350002F77012F5F5F1EC0406819B114712F777E
:1013600052501FC0406409B12F770471D1F15F5F03
:1013700000C023C0406219B12F77147191F15F5FF3
:1013800000C025C004711027515012F45D5F0000A9
:10139000115027952C3F19B1C8F61471012701503F
:1013A00027952C3FC8F64227499309B104711027AD
:1013B0004F73115027952C3FA8F64695469519B1C5
:1013C000147179F00127015027952C3F98F66B5A3C
:1013D00060F3315009B1B0F600C011E01CBB00272A
:1013E00017C03B503195C31BD04011E01CBB088196
:1013F000033CF9F00B34E9F020916E031981110FD1
:101400001213EDCF093651F10D3211F0013E39F7CB
:10141000009375033F915F914F911F910F912F9111
:101420006F91CCB3C0FD67CFDF91CF91CFBFCF918C
:10143000189520917503222369F3109173031123EA
:1014400039F534303AF13093730320936F031091E0
:1014500070033BE0311B309370031CC00091730399
:101460000130B4F40AE53091010134FD14C0009359
:101470000101C3E6D3E013C0052710E000C000005F
:101480000BB91AC0052710E0221F1DC010E021C0B3
:101490004AE502C032ED432FC4E1D0E032E01AB198
:1014A00014615C9A0BB11AB954E120E865E320FF9E
:1014B00005270BB9279517951C3FF0F66695B8F7E9
:1014C000B1F720FF05270BB9279517951C3FD0F6DC
:1014D0002795179517FF052700001C3F0BB9B0F69D
:1014E00029913A9519F70B7E10917403110FC6518B
:1014F000D0400BB911F010936E0311E01CBB0061DA
:101500001AB11B7E402F4B7E54E05A95F1F70BB970
:101510001AB94BB97FCF2EE088E190E00FB6F8946E
:10152000A895809360000FBE209360000E94570929
:10153000549A80E0815041F0A895EFE9FFE031979F
:10154000F1F700C00000F6CF54980E94220478946E
:10155000A8950E944E080E946103FACFEE0FFF1F6C
:0C1560000590F491E02D0994F894FFCF61
:02156C00FF5A24
:00000001FF
